:020000021000EC
:10000000C07702208DE901002564040079E9010030
:1000100079E9010079E9010079E9010000000000B7
:1000200000000000000000000000000095EA010050
:1000300079E901000000000001EA010079E901000E
:10004000A5EC010089350300A5EC0100A5EC010039
:10005000A5EC0100A5EC0100A5EC0100A5EC010058
:10006000A5EC0100A5EC0100A5EC0100A5EC010048
:10007000A5EC0100A5EC0100A5EC0100A5EC010038
:10008000A5EC0100A5EC0100A5EC0100A5EC010028
:10009000A5EC0100A5EC0100A5EC0100A5EC010018
:1000A000A5EC0100A5EC0100A5EC0100A5EC010008
:1000B000A5EC0100A5EC0100A5EC0100A5EC0100F8
:1000C000A5EC0100A5EC0100A5EC0100A5EC0100E8
:1000D000A5EC0100A5EC0100A5EC0100A5EC0100D8
:1000E000A5EC0100A5EC0100A5EC0100A5EC0100C8
:1000F000A5EC0100A5EC0100A5EC0100A5EC0100B8
:10010000002902D0B0FBF1F0704708B14FF0FF308A
:1001100000F01EB80029F8D00246B0FBF1F000FB59
:1001200011217047002902D090FBF1F070470028A0
:10013000C8BF6FF00040B8BF4FF0004000F008B8F3
:100140000029F4D0024690FBF1F000FB112170472A
:10015000704700BF81F0004102E000BF83F0004320
:1001600030B54FEA41044FEA430594EA050F08BF52
:1001700090EA020F1FBF54EA000C55EA020C7FEA16
:10018000645C7FEA655C00F0E2804FEA5454D4EB93
:100190005555B8BF6D420CDD2C4480EA020281EA5D
:1001A000030382EA000083EA010180EA020281EA95
:1001B0000303362D88BF30BD11F0004F4FEA0131E7
:1001C0004FF4801C4CEA113102D0404261EB4101F6
:1001D00013F0004F4FEA03334CEA133302D052427C
:1001E00063EB430394EA050F00F0A780A4F1010438
:1001F000D5F1200E0DDB02FA0EFC22FA05F2801872
:1002000041F1000103FA0EF2801843FA05F3594157
:100210000EE0A5F120050EF1200E012A03FA0EFCD6
:1002200028BF4CF0020C43FA05F3C01851EBE37100
:1002300001F0004507D54FF0000EDCF1000C7EEB1D
:1002400000006EEB0101B1F5801F1BD3B1F5001F5B
:100250000CD349085FEA30004FEA3C0C04F101047A
:100260004FEA445212F5800F80F09A80BCF1004FA3
:1002700008BF5FEA500C50F1000041EB045141EA25
:10028000050130BD5FEA4C0C404141EB0101013CEE
:1002900028BFB1F5801FE9D291F0000F04BF0146DD
:1002A0000020B1FA81F308BF2033A3F10B03B3F1AF
:1002B00020020CDA0C3208DD02F1140CC2F10C023F
:1002C00001FA0CF021FA02F10CE002F11402D8BF9D
:1002D000C2F1200C01FA02F120FA0CFCDCBF41EA69
:1002E0000C019040E41AA2BF01EB0451294330BD38
:1002F0006FEA04041F3C1CDA0C340EDC04F1140415
:10030000C4F1200220FA04F001FA02F340EA0300EB
:1003100021FA04F345EA030130BDC4F10C04C4F131
:10032000200220FA02F001FA04F340EA0300294611
:1003300030BD21FA04F0294630BD94F0000F83F45B
:10034000801306BF81F480110134013D4EE77FEA3E
:10035000645C18BF7FEA655C29D094EA050F08BF8A
:1003600090EA020F05D054EA000C04BF194610466B
:1003700030BD91EA030F1EBF0021002030BD5FEAAF
:10038000545C05D14000494128BF41F0004130BDD7
:1003900014F580043CBF01F5801130BD01F000452B
:1003A00045F0FE4141F470014FF0000030BD7FEA9E
:1003B000645C1ABF194610467FEA655C1CBF0B4699
:1003C000024650EA013406BF52EA033591EA030FB0
:1003D00041F4002130BD00BF90F0000F04BF0021A8
:1003E000704730B54FF4806404F132044FF00005DB
:1003F0004FF0000150E700BF90F0000F04BF002154
:10040000704730B54FF4806404F1320410F00045B9
:1004100048BF40424FF000013EE700BF42004FEAB4
:10042000E2014FEA31014FEA02701FBF12F07F4331
:1004300093F07F4F81F06051704732F07F4208BFE8
:10044000704793F07F4F04BF41F40021704730B5EF
:100450004FF4607401F0004521F000411CE700BF3B
:1004600050EA010208BF704730B54FF000050AE0BE
:1004700050EA010208BF704730B511F0004502D5BF
:10048000404261EB41014FF4806404F132045FEAC1
:10049000915C3FF4D8AE4FF003025FEADC0C18BF6A
:1004A00003325FEADC0C18BF033202EBDC02C2F15C
:1004B000200300FA03FC20FA02F001FA03FE40EAEE
:1004C0000E0021FA02F11444BDE600BF70B54FF0F2
:1004D000FF0C4CF4E06C1CEA11541DBF1CEA1355D0
:1004E00094EA0C0F95EA0C0F00F0DEF82C4481EA38
:1004F000030621EA4C5123EA4C5350EA013518BF58
:1005000052EA033541F4801143F4801338D0A0FB44
:1005100002CE4FF00005E1FB02E506F00042E0FBF1
:1005200003E54FF00006E1FB03569CF0000F18BFF7
:100530004EF0010EA4F1FF04B6F5007F64F540749F
:1005400004D25FEA4E0E6D4146EB060642EAC62132
:1005500041EA55514FEAC52040EA5E504FEACE2E9F
:10056000B4F1FD0C88BFBCF5E06F1ED8BEF1004FA2
:1005700008BF5FEA500E50F1000041EB045170BD1E
:1005800006F0004646EA010140EA020081EA030162
:10059000B4EB5C04C2BFD4EB0C0541EA045170BD5E
:1005A00041F480114FF0000E013C00F3AB8014F1D8
:1005B000360FDEBF002001F0004170BDC4F1000421
:1005C000203C35DA0C341BDC04F11404C4F12005A2
:1005D00000FA05F320FA04F001FA05F240EA0200FD
:1005E00001F0004221F0004110EBD37021FA04F633
:1005F00042EB06015EEA430E08BF20EAD37070BDED
:10060000C4F10C04C4F1200500FA04F320FA05F04B
:1006100001FA04F240EA020001F0004110EBD3704D
:1006200041F100015EEA430E08BF20EAD37070BDBD
:10063000C4F1200500FA05F24EEA020E20FA04F396
:1006400001FA05F243EA020321FA04F001F0004145
:1006500021FA04F220EA020000EBD3705EEA430EB6
:1006600008BF20EAD37070BD94F0000F0FD101F0E5
:100670000046400041EB010111F4801F08BF013C1E
:10068000F7D041EA060195F0000F18BF704703F05C
:100690000046520043EB030313F4801F08BF013DE3
:1006A000F7D043EA0603704794EA0C0F0CEA13559F
:1006B00018BF95EA0C0F0CD050EA410618BF52EA59
:1006C0004306D1D181EA030101F000414FF000005F
:1006D00070BD50EA410606BF1046194652EA43066D
:1006E00019D094EA0C0F02D150EA013613D195EAE1
:1006F0000C0F05D152EA03361CBF104619460AD129
:1007000081EA030101F0004141F0FE4141F4700132
:100710004FF0000070BD41F0FE4141F4780170BD22
:1007200070B54FF0FF0C4CF4E06C1CEA11541DBF87
:100730001CEA135594EA0C0F95EA0C0F00F0A7F889
:10074000A4EB050481EA030E52EA03354FEA0131B6
:1007500000F088804FEA03334FF0805545EA1313C9
:1007600043EA12634FEA022245EA111545EA106591
:100770004FEA00260EF000419D4208BF964244F128
:10078000FD0404F5407402D25B084FEA3202B61A47
:1007900065EB03055B084FEA32024FF480104FF41B
:1007A000002CB6EB020E75EB030E22BFB61A75468F
:1007B00040EA0C005B084FEA3202B6EB020E75EB22
:1007C000030E22BFB61A754640EA5C005B084FEA8A
:1007D0003202B6EB020E75EB030E22BFB61A754657
:1007E00040EA9C005B084FEA3202B6EB020E75EB62
:1007F000030E22BFB61A754640EADC0055EA060E23
:1008000018D04FEA051545EA16754FEA06164FEA65
:10081000C30343EA52734FEAC2025FEA1C1CC0D111
:1008200011F4801F0BD141EA00014FF000004FF09E
:10083000004CB6E711F4801F04BF01430020B4F15F
:10084000FD0C88BFBCF5E06F3FF6AFAEB5EB030C17
:1008500004BFB6EB020C5FEA500C50F1000041EB14
:10086000045170BD0EF0004E4EEA113114EB5C04E1
:10087000C2BFD4EB0C0541EA045170BD41F48011B4
:100880004FF0000E013C90E645EA060E8DE60CEABC
:10089000135594EA0C0F08BF95EA0C0F3FF43BAFD9
:1008A00094EA0C0F0AD150EA01347FF434AF95EA90
:1008B0000C0F7FF425AF104619462CE795EA0C0F74
:1008C00006D152EA03353FF4FDAE1046194622E741
:1008D00050EA410618BF52EA43067FF4C5AE50EA1B
:1008E00041047FF40DAF52EA43057FF4EBAE12E70B
:1008F0004FF0FF3C06E000BF4FF0010C02E000BFEC
:100900004FF0010C4DF804CD4FEA410C7FEA6C5CCE
:100910004FEA430C18BF7FEA6C5C1BD001B050EA71
:10092000410C0CBF52EA430C91EA030F02BF90EA5C
:10093000020F0020704710F1000F91EA030F58BF1B
:10094000994208BF90422CBFD8176FEAE37040F07D
:10095000010070474FEA410C7FEA6C5C02D150EA1B
:10096000013C07D14FEA430C7FEA6C5CD6D152EAD6
:10097000033CD3D05DF8040B704700BF844610469B
:1009800062468C461946634600E000BF01B5FFF79A
:10099000B7FF002848BF10F1000F01BD4DF808ED6A
:1009A000FFF7F4FF0CBF012000205DF808FB00BF3B
:1009B0004DF808EDFFF7EAFF34BF012000205DF895
:1009C00008FB00BF4DF808EDFFF7E0FF94BF0120E2
:1009D00000205DF808FB00BF4DF808EDFFF7CEFFE3
:1009E00094BF012000205DF808FB00BF4DF808ED22
:1009F000FFF7C4FF34BF012000205DF808FB00BFF3
:100A00004FEA410C7FEA6C5C02D150EA013C0AD10A
:100A10004FEA430C7FEA6C5C02D152EA033C02D1FC
:100A20004FF0000070474FF0010070474FEA41025D
:100A300012F5001215D211D56FF47873B3EB625230
:100A400012D94FEAC12343F0004343EA505311F057
:100A5000004F23FA02F018BF404270474FF00000E9
:100A6000704750EA013005D111F0004008BF6FF027
:100A7000004070474FF00000704700BF4A0011D29D
:100A800012F5001211D20DD56FF47873B3EB6252E8
:100A90000ED44FEAC12343F0004343EA505323FAF4
:100AA00002F070474FF00000704750EA013002D169
:100AB0004FF0FF3070474FF0000070474FEA41029F
:100AC000B2F1E04324BFB3F5001CDCF1FE5C0DD9AC
:100AD00001F0004C4FEAC0024CEA5070B2F1004FF6
:100AE00040EB830008BF20F00100704711F0804FF9
:100AF00021D113F13872BCBF01F00040704741F4BE
:100B000080114FEA5252C2F11802C2F1200C10FAC1
:100B10000CF320FA02F018BF40F001004FEAC123A5
:100B20004FEAD32303FA0CFC40EA0C0023FA02F349
:100B30004FEA4303CCE77FEA625307D150EA01331F
:100B40001EBF4FF0FE4040F44000704701F00040EF
:100B500040F0FE4040F40000704700BF80F00040CD
:100B600002E000BF81F0004142001FBF5FEA410385
:100B700092EA030F7FEA226C7FEA236C6AD04FEA85
:100B80001262D2EB1363C1BFD218414048404140CA
:100B9000B8BF5B42192B88BF704710F0004F40F47C
:100BA000000020F07F4018BF404211F0004F41F498
:100BB000000121F07F4118BF494292EA030F3FD064
:100BC000A2F1010241FA03FC10EB0C00C3F1200377
:100BD00001FA03F100F0004302D5494260EB400006
:100BE000B0F5000F13D3B0F1807F06D340084FEA71
:100BF000310102F10102FE2A51D2B1F1004F40EB66
:100C0000C25008BF20F0010040EA030070474900CD
:100C100040EB0000013A28BFB0F5000FEDD2B0FA6A
:100C200080FCACF1080CB2EB0C0200FA0CF0AABF8D
:100C300000EBC25052421843BCBFD040184370472B
:100C400092F0000F81F4000106BF80F40000013231
:100C5000013BB5E74FEA41037FEA226C18BF7FEA08
:100C6000236C21D092EA030F04D092F0000F08BF4A
:100C70000846704790EA010F1CBF0020704712F031
:100C80007F4F04D1400028BF40F00040704712F170
:100C900000723CBF00F50000704700F0004343F0D5
:100CA000FE4040F4000070477FEA226216BF08460B
:100CB0007FEA23630146420206BF5FEA412390EACE
:100CC000010F40F4800070474FF0000304E000BFC4
:100CD00010F0004348BF40425FEA000C08BF704775
:100CE00043F0964301464FF000001CE050EA010239
:100CF00008BF70474FF000030AE000BF50EA01024E
:100D000008BF704711F0004302D5404261EB41013A
:100D10005FEA010C02BF84460146002043F0B6435F
:100D200008BFA3F18053A3F50003BCFA8CF2083A84
:100D3000A3EBC25310DB01FA02FC634400FA02FC8D
:100D4000C2F12002BCF1004F20FA02F243EB020094
:100D500008BF20F00100704702F1200201FA02FCF6
:100D6000C2F1200250EA4C0021FA02F243EB0200E9
:100D700008BF20EADC7070474FF0FF3C06E000BF80
:100D80004FF0010C02E000BF4FF0010C4DF804CD14
:100D90004FEA40024FEA41037FEA226C18BF7FEA24
:100DA000236C11D001B052EA530C18BF90EA010F26
:100DB00058BFB2EB030088BFC81738BF6FEAE170B5
:100DC00018BF40F0010070477FEA226C02D15FEA51
:100DD000402C05D17FEA236CE4D15FEA412CE1D0BD
:100DE0005DF8040B704700BF844608466146FFE784
:100DF0000FB5FFF7C9FF002848BF10F1000F0FBD66
:100E00004DF808EDFFF7F4FF0CBF012000205DF85E
:100E100008FB00BF4DF808EDFFF7EAFF34BF0120E3
:100E200000205DF808FB00BF4DF808EDFFF7E0FF7C
:100E300094BF012000205DF808FB00BF4DF808EDCD
:100E4000FFF7D2FF94BF012000205DF808FB00BF30
:100E50004DF808EDFFF7C8FF34BF012000205DF812
:100E600008FB00BF4FEA40024FEA41037FEA226CD1
:100E700002D15FEA402C08D17FEA236C02D15FEAFD
:100E8000412C02D14FF0000070474FF00100704735
:100E90007BB972B90029BEBF00204FF0004106E0C7
:100EA00008BF00281CBF6FF000414FF0FF30FFF774
:100EB0004FB9ADF1080C6DE904CE002909DB002B18
:100EC0001ADB00F09CF8DDF804E0DDE9022304B051
:100ED0007047404261EB4101002B1BDB00F08FF8B3
:100EE000DDF804E0DDE9022304B0404261EB41019A
:100EF000524263EB43037047524263EB430300F0FB
:100F00007EF8DDF804E0DDE9022304B0404261EB45
:100F100041017047524263EB430300F070F8DDF883
:100F200004E0DDE9022304B0524263EB430370475F
:100F300053B94AB9002908BF00281CBF4FF0FF3140
:100F40004FF0FF30FFF704B9ADF1080C6DE904CEA6
:100F500000F055F8DDF804E0DDE9022304B0704745
:100F6000D0B50C4B002206460F46FFF7AFFAFFF74D
:100F700085FD0446FFF730FA074B0022FFF7A6FA7B
:100F800002460B4630463946FFF7E8F8FFF776FD94
:100F90002146D0BD0000F03D0000F04110F8012BCB
:100FA00011F8013B012A28BF9A42F7D0D01A7047A6
:100FB000034611F8012B03F8012B002AF9D17047E1
:100FC000034613F8012B002AFBD1181A0138704789
:100FD00038B50022002304460D46FFF7E9FC28B986
:100FE00020462946BDE83840FFF7BABF204605F144
:100FF0000041FFF7B5FF404261EB410138BD2DE9EB
:10100000F04786468C460846089E154674461946A3
:10101000002B40F0C2808542B2FA82F245D94AB133
:10102000C2F1200300FA02FC2EFA03F3954043EAD2
:101030000C0C94404FEA154EA8B2BCFBFEF8230CF2
:101040000EFB18CC08FB00F943EA0C43994528D95C
:10105000EB1808F1FF3704D2994502D9A8F102072D
:101060002B44A3EB0903A4B2B3FBFEFC0EFB1C3321
:101070000CFB00F044EA0344A04214D92C190CF1F3
:10108000FF3304D2A04202D9ACF102032C44241A4B
:1010900043EA07401EB1D440002334607360BDE8CA
:1010A000F0874746DDE76346F1E792BB431B01212A
:1010B0004FEA154EAFB2B3FBFEFC200C0EFB1C3307
:1010C0000CFB07F840EA0343984562D9EB180CF192
:1010D000FF3004D2984502D9ACF102002B44A3EBB7
:1010E0000803A4B2B3FBFEFC0EFB1C330CFB07F79A
:1010F00044EA0344A7424ED92C190CF1FF3304D221
:10110000A74202D9ACF102032C44E41B43EA00409D
:10111000C0E7C2F1200320FA03F1954090402EFA77
:1011200003F303434FEA154EAFB2B1FBFEFC0EFBD7
:101130001C10190C0CFB07F841EA0041884504FA21
:1011400002F422D969180CF1FF3004D2884502D983
:10115000ACF102002944A1EB08019BB2B1FBFEFCFB
:101160000EFB1C110CFB07F743EA01439F420ED90B
:10117000EB180CF1FF3104D29F4202D9ACF102010D
:101180002B44DB1B41EA004192E76046E3E76146FE
:10119000F7E76046A3E76346B7E7834206D916B987
:1011A000002108467BE7C6E900E0F9E7B3FA83F7D8
:1011B0008FB9834201D3724508D8BEEB020460EBBD
:1011C000030301209C461EB9002168E73846FAE770
:1011D000C6E9004CF8E7C7F1200CBB4022FA0CF43A
:1011E0001C432EFA0CF120FA0CF3B84001434FEAED
:1011F00014490EFA07F5B3FBF9F81FFA84FE09FB50
:1012000018300B0C08FB0EFA43EA00439A4502FA29
:1012100007F240D9E31808F1FF3004D29A4502D909
:10122000A8F102002344A3EB0A0389B2B3FBF9F847
:1012300009FB183308FB0EFE41EA03418E452CD909
:10124000611808F1FF3304D28E4502D9A8F10203D8
:10125000214443EA0040A0FB0298A1EB0E01414566
:10126000CE46434602D306D14D4504D2B9EB020E19
:1012700068EB04030138002EA6D0B5EB0E0261EB3B
:10128000030101FA0CFC22FA07F34CEA0303F940CC
:10129000C6E9003198E74046C5E74346D9E7000074
:1012A0002DE9F047064688B00F46904637F02CF9F6
:1012B0004FF47A73A0FB034503FB0155E40B012FA8
:1012C00044EA45444FEAD53507D1294922462B4601
:1012D000304634F058F8002012E0D8F80470254861
:1012E0003946FFF75BFE70B123483946FFF756FEDB
:1012F00048B1304621493A4634F061F86FF00400B5
:1013000008B0BDE8F0872046294617A3D3E900239B
:10131000FFF7BEFD05460C4610461946184A002345
:10132000FFF7B6FD80460F46104619464EF660227E
:101330000023FFF7ADFD82468946104619464FF45B
:101340007A720023FFF7A4FDCDE902A9CDE90623B7
:10135000CDE90401CDE900870A492A4623463046F3
:1013600034F011F8B7E700BF005C2605000000006C
:10137000F9D904000ADA04000DDA040016DA0400D0
:1013800080EE36002EDA04002DE9F843D0E9073864
:10139000856903EB08042F34A5420F46164619D879
:1013A000DFF87080A3FB080117A3D3E90023FFF740
:1013B000BFFD0346601BA0FB080123F07F4412A37E
:1013C000D3E90023FFF7B4FD20F07F403C6030609C
:1013D000BDE8F883DFF83C900BA3D3E90023A5FB1D
:1013E0000901FFF7A5FD20F07F4409480A2106A363
:1013F000D3E90023E8FB0901FFF79AFD20F07F40C5
:101400003C603060BDE8F8838D49FD1A070000009C
:1014100000166BF100CA9A3B154B164A30B44FF0D8
:10142000FF31154C196015492060154B4FF0FF3402
:1014300041F6FF75C1E90045002000219FED0A7BC0
:10144000C3E900010F4C1049104D114800230B60F7
:1014500084ED007BC2E900330E492B6003600B6012
:1014600030BC11F067BF00BF1F000000000000008B
:10147000C0740020A8740020A0740020C0000020C8
:10148000C80F0020B8000020B87400209C74002011
:10149000B4740020B07400202DE9F04F8DB09A464E
:1014A000179C9DF85890636C05460E46904653B1C4
:1014B000B4F884301BB1B4F882209A4278D2D4F8C0
:1014C0008820002A77D14FF6FF739A4520D02778DD
:1014D0000137FFB22770002F78D06F496F4BC1F8EA
:1014E000048004F11C000022C86081F80A900D609D
:1014F000A1F808A09960012011460EF043F90028D8
:1015000073D1636CC4F89C5013B1204617F036FCBD
:1015100094F8245015F001054AD1614A614B1178C5
:101520001B788B4277D04FF6FF739A45D4F88880AA
:10153000B4F8829015BF0AF101074FF0000ABFB25C
:101540005746B8F1000F30D0B9F1000F2DD0626FBF
:101550000AF1010A40F271211FFA8AF301FB02FA33
:101560000AFB03F30993504B4FF0070BA6FB030153
:101570000BFB061146A3D3E90023FFF7D9FC099A18
:10158000494B1618A5FB03010BFB051140A3D3E93A
:101590000023FFF7CDFC50443044804586BFA8EBC4
:1015A0000606C4F88860C4F888A04F44A4F8827086
:1015B0000DB0BDE8F08F616F40F27123A1FB031302
:1015C000914273F10003FFF47EAFF1E7374A3849E7
:1015D000384840F64A1332F0E0FF87F31188BFF332
:1015E0006F8F0323184602DF77E7304A32493148CC
:1015F00040F66E1332F0D1FF002383F31188BFF35E
:101600006F8F0323184602DF636CC4F89C50002BD5
:101610007FF47BAF7CE7013304210BA8137022F029
:10162000E5FA0B9B25490694A1FB0321581A244A8D
:10163000009501EB50012348A21AA0FB0202090AFF
:1016400040F24710D20900FB113302321E490591C6
:101650000133CDE90355CDE90155D2B20121284628
:101660000B930FF097FD10F0FD0F0DD00F4A1749A7
:10167000104840F2BB7332F090FF85F31188BFF33E
:101680006F8F0323184602DF0B9D4CE7AFF30080FA
:1016900000CA9A3B00000000E4760020F00200201F
:1016A000E7980020E69800208D49FD1A9CB10400BF
:1016B000A8B204007CAA040070AC040021F1D4900C
:1016C000D00F0020CDCCCCCC356D0200ACB20400E4
:1016D000002900F072812DE9F04F91B0002840F010
:1016E000B882B74C174694F88C2012F001051E46BC
:1016F00040F0B98294F82500FF2300F0030084F83D
:10170000273021F0CBF994F88C00410700F10681D5
:1017100094F8352094F8293004EB820204EB83031B
:10172000D2F83880D3F82CA0B8F1000F00F0DC809C
:101730004146504616F040FB0546002840F03981EE
:101740009AF8003013F00E0F40F04881236A002B06
:1017500040F02E8110F0DCFE0546002800F0B38238
:1017600010F0E2FE0A90002800F0AA8219F074FC42
:101770008346002800F0A182D0F894004FF6FF7253
:101780000BF11C03ABF830200B93002800F0D08243
:101790000BF188020BF184010DF06EFF9BF89A208B
:1017A00022F007028BF89A200022CBF89420ABF8A5
:1017B00098209AF8002002F00F02072A00F0A88271
:1017C0009BF8822022F0770242F011028BF88220EF
:1017D000012211467B48D0F801C0CBF8AFC1D2003E
:1017E000CBF8B5C110F801CB42EA01219BF8AE213C
:1017F0000CF0010C6CF300026CF341028BF8AE218B
:101800008288ABF8B321ABF8B921BBF8822022F46F
:10181000E16211439BF84320ABF8821002F03F02D3
:1018200062F07F028BF843209BF848207F214FF025
:10183000000922F00F028BF8DE104FF4C0218BF864
:101840004820CBF89C115846CBE915998BF8459068
:10185000ABF83690CBF83A90CBF85C90ABF8A2910D
:10186000ABF898911CF000FC8BF86091CBF86451B8
:1018700019F0F6FF9BF8A81160F302018BF8A8118C
:1018800019F0F4FF9BF8A81160F3C5018BF8A811BB
:101890009BF8941169F341018BF894119AF8002098
:1018A00002F00F02072A0ABF94F825100121490906
:1018B00058461AF089FC0BF1E0001CF07DF90A9BF8
:1018C000236700220B9BE5662362CBE90522CBF858
:1018D0001CB08BF8002022F0E9FC002800F0838087
:1018E00015F0B0FB032564E09AF8003003F00F0315
:1018F000072B5DD0344822F093FEC0B2002840F0A0
:10190000E28194F8353004EB8303D3F83880042364
:1019100088F80030062388F8013009E7C0F3C000DA
:101920002A4604F18D0121F099FAFF2884F8270056
:101930003FF4EEAE284621F0F7F8E9E6234B099391
:1019400000200EAA186002250892214E214A059215
:101950000321CDE902000694CDF81080CDF8048073
:101960003B46009007962A460E950FF0B3FB0EA952
:1019700010F096FEC0B90EAA174908924AF2D83262
:1019800000920591CDE903000321CDE901000796FE
:101990003B46069401220E950FF068FB0EA910F04D
:1019A0007FFE002800F03F81236A0BB115F04AFB4F
:1019B0000C25284611B0BDE8F08F15F087BB00BF9D
:1019C000D00F00204DF00400041000200477002008
:1019D000C915020099140100956B020003F00F0372
:1019E000072B00F0AA81C24B1B78022B00F0AB81C1
:1019F000002323640026374694F8242094F82630E8
:101A0000A4F88460C2F34202012100250DF13500E3
:101A100094F82560C4F888708DF8352003EA010732
:101A2000A4F882500DF0C6FFC6F3820602460028D5
:101A3000BAD0009733464146504615F049F8AD49B3
:101A4000AD4B2570A0FB0101C0184FF0310341F1EF
:101A50000701A360C4E90555A3A3D3E9002365608A
:101A6000E560FFF765FAB4F8749020610FF0DAFCD6
:101A700000F11807B9F1000F08D19AF8005005F0ED
:101A80000F05A5F10105B5FA85F56D0994F8243027
:101A9000D4F8108065F3000313F0010584F82430B6
:101AA0007FF44CAFA36C002B00F0CB80D3F800A0E8
:101AB0009AF8523003F0030BBBF1010F40F0C180E4
:101AC0000DF137030EA901930DF136032A460A9151
:101AD00000938A480B46202100F06AFA0546002848
:101AE0007FF467AFDDF83910504617F09DFF666C44
:101AF000002E00F0568136680A9908F102033B4433
:101B000030460E9300F0BCF95F2211460B90304630
:101B100017F02AF9774974A3D3E90023A0FB010148
:101B2000FFF706FA0E9B0B9902330B4420F07F401F
:101B30002A465146C518714801F072F92A460346F3
:101B400051466E4801F0B4F900287FF42DAF636C64
:101B50009DF837205A759DF8363084F829305D4657
:101B6000636F94F8802040F27121A3FB0131002AB9
:101B700040F0FE8042F6DC32981841F1000140F25C
:101B8000E2420023FFF7D4F980B2B0870B9A0E9996
:101B9000304600F0BDF900287FF406AF4FF0010B8E
:101BA0000A9B08935648574BCDF8108008F247120D
:101BB000069491211A600993A9FB000301FB0931E6
:101BC000514B0793514B05934FF6FF734FF00008AD
:101BD0004FF00209039344A3D3E90023CDF8088012
:101BE000CDF83890FFF7A4F9032101903B464A460F
:101BF000CDF8008040460FF06DFA0A9910F050FDC4
:101C000000287FF4D1AEBBF1000F0CD096F84E3017
:101C100043F0010386F84E302DB19AF8523043EA72
:101C200009038AF8523094F88C30002043F0010305
:101C300084F88C3018F03AFD80B9012020F010FFB4
:101C40000CE0666C002E40D10EABB246B3460A9350
:101C5000A6E7274B1B78022B3FF4AAAE00252846A7
:101C600011B0BDE8F08F224B1B78022BF6D194F80F
:101C7000352094F8293004EB820204EB8303916B46
:101C8000D86A16F099F8054600287FF492AE236CC6
:101C9000002B3FF48DAE1A7902F0FF014AB942F2EF
:101CA000107207FB02F2A4F88210A4F88460C4F852
:101CB00088201B79002BD1D07AE60A9810F03AFCE4
:101CC000284610F02BFC072573E608F1020336685E
:101CD0003B440E930EAB194630460A9300F0D0F801
:101CE0004FF0000A0B903BE78D49FD1A07000000FA
:101CF000E598002000CA9A3B8C49FD1AD00F0020BD
:101D0000002AE78404770020C91502009914010015
:101D100094F825109BF88220490961F3020261F3CF
:101D200006128BF8822094F8262002F0010251E579
:101D30000BF18C00CBF894002AE59AF802305A0691
:101D40007FF551AE02E510F0E3FB0546E8B110F077
:101D5000EBFB00B300230560037194F8243020648A
:101D6000DB073FF547AE42F2107303FB07F743E68C
:101D700002FB01110132A2FB0303194440F2E242CB
:101D80000023FFF7D5F880B2FFE6236A002B9AD034
:101D900015F058F997E7236A002B91D015F052F906
:101DA0008EE7B346FCE600BF2DE9F04190F8243001
:101DB00090F8257090F826808AB00D46C3F3420350
:101DC000044601210DF1230016468DF823300DF055
:101DD000F1FDC7F3820708F0010802463B46314691
:101DE0002846CDF8008014F073FE1F491F4AA0FB5F
:101DF0000131981841F1070119A3D3E90023FFF736
:101E000097F823699842054622D21B1A00220192B4
:101E1000174A0293174BA21AA3FB02320221D209DE
:101E200000230A4409AE099113490591CDE9033312
:101E30000321D2B20696009318460FF0ABF9314653
:101E400010F02EFC40B9256100200AB0BDE8F081F9
:101E5000FAD9C21A0023DAE70C200AB0BDE8F081F3
:101E60008D49FD1A0700000000CA9A3B8C49FD1AF3
:101E7000D00F0020CDCCCCCCC91502000000000052
:101E80002DE9F04182B004461F4E204F884616F0DF
:101E900025F9072500236360E36029463346E0FB0C
:101EA00007313122A260184615A3D3E90023FFF7BA
:101EB0003FF894F8313020F07F4004EB8303206139
:101EC000596B5F231A46204616F0A6F82946E0FB18
:101ED00007610BA3D3E900233046FFF729F801A9D6
:101EE00020F07F4020F030F818B9019B0233C8F889
:101EF0000030002002B0BDE8F08100BFAFF30080E9
:101F00008D49FD1A070000008C49FD1A00CA9A3B52
:101F10002DE9F04700268CB08846C0E905662049C7
:101F200006701746502204460DF086FB0546A08F2A
:101F30001C4940F2E24202FB00F002230B93A0FB9B
:101F4000010115A3D3E90023FEF7F2FF0DF12C0ADE
:101F5000CDF820A00694194623691F44124B07931D
:101F6000124B05938146002310464FF47A72CDE957
:101F70000367FEF7DDFF0335EDB2CDE9019043467F
:101F80002A460096304603210FF070F8514610F0B3
:101F900087FB0CB0BDE8F0878D49FD1A07000000F3
:101FA0005477002000CA9A3BC9150200198102002B
:101FB0002DE9F04FA5B00C461E4640F201232E99A4
:101FC0000E92A3432F9A0F910546109200F09F8125
:101FD00095F8293005EB8303D3F82CA09AF800700C
:101FE00007F00F0204F40073072A0C9309920FD034
:101FF0002BB90C230993099825B0BDE8F08FD6F8CA
:1020000001203178284625B0BDE8F04F15F028BFF3
:102010000AF104019AF802300B910C9913F03F0277
:1020200018BF9AF8032011B17F2B00F292810F990B
:10203000089205F1280022F0A9FB9AF80010037815
:10204000024601F00F0123F03F030B4302F8023B6D
:1020500081469AF8023099F8021018929B0963F3AE
:10206000871189F80210696C089A05F11C004FF07D
:102070000008002900F0EE824B7D01EB8303986994
:102080000B681293C3780D900230169003F0010094
:10209000159001F1140010990A93089222F076FB32
:1020A000804699F8000098F800100D9B089A00F0FF
:1020B0000F0021F03F01014388F80010197898F8CB
:1020C0000000C1F3801161F3861088F800001978D0
:1020D0000A9BC909C0B261F3C71088F8000099F8DB
:1020E000021098F80200890961F3871014F00101C9
:1020F00088F802004FF0010B02F0010040F0178158
:10210000002800F05D819AF8000098F800C0C0F344
:10211000801060F3861C88F800C099F8000061F315
:10212000861089F800000AF10A000B901598002823
:1021300040F05A810D980430089003F00200179087
:10214000900740F121810B9998F800C006310B915E
:102150009AF800104046C90961F3C71C00F810CB7B
:102160004FF0030B99F800106FF3C71189F80010B6
:10217000179911B108990631089112F008011C91C4
:1021800002D00B9902310B91811C0A9114F00801C5
:1021900000F0F88002213170D6F801101B91C6F8CA
:1021A000010005364BF0080113F008078B461D9718
:1021B00002D0089F0237089712F010071E9702D02E
:1021C0000B9F03370B974FF018078DF8687009F1D4
:1021D0000907119703F010071397E70640F1C7802E
:1021E000871C41F0100B0321C6F8017031700536D1
:1021F0001399002900F0C38000211F910899033131
:1022000008911BF0100F1CBF05300A9003F020004E
:10221000A7065FFA8BF1149040F19E800A98C6F8E9
:1022200001004BF02001122030708B460536C9B2F8
:102230001498002800F09880002020900898123010
:102240000890890602D50A9912310A91520610D5D2
:102250000B9A01320B9295F8252002F01C02102AED
:1022600000F017824FF058028DF8682009F10A0239
:1022700011925B0604D5089B013308934BF0400B89
:102280005FFA8BF319931BF04003219302D00A9B52
:1022900001330A93119B189A9B1ADBB2022B03D8C5
:1022A00009F1030311930123089A1699501AC0B239
:1022B000022803D80D9A0332089201200D9A517812
:1022C0008142C0F08F810A9F08F10202BA1AD2B28D
:1022D000022A03D808F103020A9201220C9F002F60
:1022E00000F08680089C081AD6F80110C6F8014054
:1022F0003478C0B230700536002C40F0818100295E
:1023000000F0E98127460C94A446204684E0B24AB6
:10231000B249B34840F2FB5332F03FF9002383F354
:102320001188BFF36F8F0323184602DF50E616F8BB
:1023300001EB98F800C06EF3861C88F800C099F88D
:1023400000C06FF3861C89F800C000283FF4EEAE91
:10235000E9E6122309934EE60E9880063FF568AF32
:102360001498002840F05E811498209069E70E9F31
:10237000FF063FF53DAF139F002F40F04E811399AC
:102380001F913EE71B910DE708F10A0000297FF439
:10239000E9AE179F002F00F039810D9898F800C022
:1023A0000078C00960F3C71C40464FF0030B00F8EB
:1023B00010CB99F800C061F3C71C89F800C0D9E6BA
:1023C0001598002800F00E810D9898F800C000784C
:1023D000C0F3801060F3861C88F800C099F80000F4
:1023E00061F3861089F800000D980A300890A4E681
:1023F000670500F1FA800E9CA40500F17281DDF8FA
:1024000030C00C1A0899E4B2674604EB0C0EBEF11A
:102410001F0F20463FF7EFAD104460445F2800F3E4
:10242000088199F8020089F80130013B63F3050047
:1024300089F8020098F80230501E60F3050388F80E
:1024400002303E463B190A9F1A4488F8012038465C
:10245000224636F033FA0C9B23B13246194638191E
:1024600036F01EFA98F802309A0600F0B1801A9BF6
:102470005B0640F121810B9A119912F8013C01F899
:10248000013C531E0B934B1E1193149B13B1089BDD
:10249000123B0893199B9F0602D50A9B123B0A9395
:1024A000209B23B10A981946122236F007FA1E9B88
:1024B00013B10B9B033B0B93119E95F8253016F837
:1024C000032C6FF3050206F8032C5C0921F040FF92
:1024D00032288CBF0020012094FAA4F3002CB3FA18
:1024E00083F308BF4FF0FF335B0106F8013C16F899
:1024F000033C60F386136FF3C71306F8033C002315
:1025000006F8023C139B13B1089B033B0893199BED
:10251000DE0602D50A9B033B0A931F9B23B10A9850
:102520001946032236F0CAF91C9B13B10B9B023BE0
:102530000B931D9B13B1089B023B08931B9B002B25
:1025400000F00B811B9A537812781B0203F470631E
:102550001A431198D1B200F8051C95F87E30C3F3E8
:1025600003031B0103EB122300F8043C0A9800F854
:10257000021C95F87E30C3F303031B0103EB122307
:1025800000F8013C199B9D0700F186800238199BD9
:10259000DC0709D5159B002B00F0F680089B991FDE
:1025A0000638062236F08AF999F8023099061CBFDF
:1025B0009DF8683089F8033098F802309A06129B2B
:1025C00018BF88F803B093F84E30DB0700F18F8016
:1025D000002309930FE500BF88B30400FCB3040097
:1025E0007CAA04001F23099305E5081A3178C4B2B8
:1025F000D6F801000C900F468C460536089904E782
:102600004FF0000C6746CDF830C0FEE699F800C0E8
:1026100061F3C71C89F800C0AFE541F0100B0899C1
:102620001F91EBE54BF02001089820908B46C9B232
:1026300004E6A2F15F033A461A4413462344CA450E
:10264000337000F09C800D9B984500F093804523EB
:102650000993D0E416F04CF9089A1290002800F083
:102660009F801299CDF8548091F8313001EB8303AB
:102670000121586B0D90074617F8023B41701299E3
:10268000169703F03F03037080F803801C31434624
:10269000FFE44BF0400BECE5179B002B77D0089B39
:1026A000063B08930A991A6841F8082C9B8821F880
:1026B000043CA1F108006AE7219B002B3FF4E5AE42
:1026C000089A0A9912F8013C01F8013C531E08933C
:1026D0004B1E0A93D9E60F46044608990C97BC4650
:1026E00093E60C9C21462746A446204694E6129C7D
:1026F000204615F0F3FC364A364B0721E0FB023149
:10270000184631A3D3E90023FEF712FC256920F017
:102710007F44AC423FD22E1B0025129F2E4902233C
:102720005022384623930CF087FF00232B49019554
:10273000C21C23AD0591CDE9033303210296D2B229
:102740000093184606950EF025FD29460FF0A8FFC8
:1027500000287FF44EAC3C613AE795F87E30204982
:1027600003F00F0331F81320501C21F81300C2F3BB
:102770000B02EEE6109A6B6C12785A7567E70F9BA6
:102780001B7885F829305EE70B9B991F08E70B9BA8
:10279000063B0B9386E77FF61BAF651B0026BCE765
:1027A000CA457FF428AC0F4A0F49104840F22E6307
:1027B00031F0F3FE129B83F31188BFF36F8F032375
:1027C000184602DF17E400BF8D49FD1A070000001C
:1027D00000CA9A3B8C49FD1A54770020C9150200A3
:1027E0003077002088B304004CB404007CAA0400B5
:1027F00070B590F803C01CF0010F14BF00F10A047B
:10280000041D1B481CF0020F15461E464FF0070220
:10281000A1FB000318BF063402FB01311CF0080FB6
:1028200011A3D3E9002318BF0234FEF781FBAD1BCF
:1028300010492844A1FB00310D09490C04D00E4B6E
:10284000A3FB003001214509A2782078657022F0B1
:102850001F02C5F3042361F3C71013432070A37054
:10286000204670BDAFF3008000CA9A3B0000000014
:102870008D49FD1A89888888B5814E1B00000000AB
:102880002DE9F04F91B0D0F844B0B34900240E9434
:10289000DBF8003009930646502218460CF0CCFEB7
:1028A000D6F89CA00C94FF23C51CEDB28DF82F30F8
:1028B0005346CDF834A00124AA460DF13C090DF190
:1028C00038080CAF1D460DE00D9BAB4203D0002C29
:1028D0002FD0013CE4B29DF82F30FF2B3DD09A451C
:1028E0004ED00D9D9D4B059300200221CDE900782F
:1028F000CDE90300CDF8189002900DAB0DF12F0239
:102900000F910EF029FD022800F0F6800F9B002B9E
:10291000DAD0934A9349944840F6AF4331F03DFEF4
:10292000002383F31188BFF36F8F0323184602DF60
:10293000CAE78E498A4A8C4840F6B84331F02DFEEA
:1029400084F31188BFF36F8F0323184602DF9DF8CD
:102950002F30FF2B4FF0FF04C1D18549804A8248B8
:1029600040F6BA4331F019FE002383F31188BFF318
:102970006F8F0323184602DF9DF82F309A45B0D1A0
:102980000E9D7C4A0C9FA5F57423A3F5107393420A
:1029900007D905F1E875013F05F5D4350C9705F524
:1029A000A575754BCBF80C70A3FB0535AD0CCBF8BA
:1029B000105096F8282096F829100E958A42D3B226
:1029C00004D00133DBB2022B08BF002306EB8303E4
:1029D00096F82520D3F82CA0BBF808909AF801307F
:1029E000C2F38202032A40F29380DC0096F826307C
:1029F00003F001035B002B3401339C4004F5BC74ED
:102A0000A4B25E4B4FF00708A7FB030108FB0711B8
:102A10004DA3D3E90023FEF78BFA594A05EB000CCE
:102A2000A2FB0C1204F5967422F00F01A3B2A1EBE5
:102A30001212B3EB420F22D9099A5248938F40F2F7
:102A4000E24202FB03C5A5FB000141A3D3E9002339
:102A5000FEF76EFA494B20F07F47A7FB0301CBF846
:102A60000C7039A3D3E9002308FB0711FEF760FAC5
:102A700009F101092D1ACBF810501FFA89F92A46DD
:102A8000394600235046FFF7B3FEDBF80C300999B6
:102A9000099D0133CBF80C3091F84D2091F84C3062
:102AA000934202EB420305EB430318BF81F84C202D
:102AB00093F84530062101FB02524032E98F04466B
:102AC00003F03F0348461FF005FB237860F305033E
:102AD00023700EF0A7FC0D990EF0A6FCD6E901219B
:102AE000F36891422CBFC3EB0103C3EB020398428E
:102AF00015D211B0BDE8F08F0F9B022B7FF406AF0B
:102B0000022100200EF076FC0F9B022BF8D0FDE690
:102B1000D4180934E4005210D440A4B271E7104A2A
:102B20001949114840F6065331F037FD002383F36D
:102B30001188BFF36F8F0323184602DF11B0BDE881
:102B4000F08F00BFAFF3008000CA9A3B0000000086
:102B50008D49FD1A070000005477002015810200FE
:102B600088B3040070B404007CAA040078B40400A4
:102B7000A8B40400BFBDF07F83DE1B438D49FD1A5E
:102B80008988888800CA9A3BCCB404000000000001
:102B90002DE9F04F91B0D0F848B0099000250E957E
:102BA000DBF8003092490893184658220CF044FD97
:102BB000FF23061DCDE90C55F6B28DF82D30042407
:102BC0000DF13C0A0DF12E090DF138080CAF0DE0A6
:102BD0000D9BAB4203D0002C2FD0013CE4B29DF8FA
:102BE0002D30FF2B3DD09E424ED00D9D814B059345
:102BF00000200221CDE90189CDE90300CDF818A01C
:102C000000970DAB0DF12D020F910EF0A5FB0228E0
:102C100000F0D7800F9B002BDAD0774A77497848AD
:102C200040F6AB2331F0B9FC002383F31188BFF3E6
:102C30006F8F0323184602DFCAE772496E4A704855
:102C400040F6AD2331F0A9FC84F31188BFF36F8FF8
:102C50000323184602DF9DF82D30FF2B4FF0FF04B1
:102C6000C1D16949644A664840F6AF2331F095FC0A
:102C7000002383F31188BFF36F8F0323184602DF0D
:102C80009DF82D309E42B0D10E9B60490C9FA3F55C
:102C90007422A2F510728A4207D903F1E873013F4A
:102CA00003F5D4330C9703F5A573089A5849526D70
:102CB000A1FB03139E0C5549A2F57423A3F51073D1
:102CC0008B4207D902F1E872013702F5D4320C9732
:102CD00002F5A572099B596C4D4B487DA3FB02324E
:102CE000950C0A7D0E958242D3B204D00133DBB23B
:102CF000022B08BF002301EB83018C69E378D8071E
:102D000048BF0A34434858BF0434990748BF0634C3
:102D10001A0748BF02340721DB06A7FB000301FBAB
:102D2000073131A3D3E9002348BF0334FEF700F98C
:102D3000731B1844B0F5161F374A28BFA0F51610AC
:102D4000A2FB00122CBF40230023550C4FEA1211A6
:102D500043D0324AA2FB0020C0F34712C0F34430F4
:102D60000343203363702270BBF81010BBF814309B
:102D7000BDF82E200B44134423829BF824209BF89B
:102D800025108A429BB206D0BBF826001B1A13F40A
:102D9000004F08BF0A461821062313FB02130BEB52
:102DA00003025BF803306360137903F01F0323729F
:102DB00021F0CCFA237A43EA4013237211B0BDE824
:102DC000F08F0F9B022B7FF425AF022100200EF025
:102DD00011FB0F9B022BF8D01CE743EA1233DBB246
:102DE000CAB2BFE7AFF3008000CA9A3B0000000000
:102DF000C8770020498E0200ECB4040070B40400CF
:102E00007CAA040078B40400A8B40400BFBDF07F1D
:102E100083DE1B438D49FD1A89888888B5814E1B46
:102E200038B50023C1E905330C460B708AB3256A17
:102E300053789278687A3E33C2F305029B1A7F2852
:102E40004FEA5011DBB21CD9AA7A02F00102DB0072
:102E500052002B330132934003F27D431248134A50
:102E60000721E3FB002100253123A36010466560A4
:102E70000BA3D3E90023E560FEF75AF8206128464A
:102E800038BD0B440933DB004910CB4003F2053356
:102E9000E4E791F8453001EB83039A6CC7E700BF84
:102EA0008D49FD1A0700000000CA9A3B8C49FD1AA3
:102EB0002DE9F047B1F850500E4640F2E2418CB097
:102EC000904601FB05F558221D4930461F460CF07F
:102ED000B3FB04461B4802230B93A5FB000116A37A
:102EE000D3E90023FEF724F80DF12C0ACDF820A039
:102EF0000696194633691F44134B0793134B0593EA
:102F000000258146002310464FF47A72CDE903571D
:102F1000FEF70EF80434E4B2CDE9019043462246B0
:102F20000095284603210EF0A1F851460FF0B8FB9A
:102F30000CB0BDE8F08700BF8D49FD1A0700000006
:102F4000C877002000CA9A3BC9150200B98E02005A
:102F5000F0B58A784B7803F13E01C2F30503C91A34
:102F60008BB0C9B2044616F02FF91D491AA3D3E954
:102F70000023A0FB0101FDF7DBFF266920F07F4560
:102F8000AE4220D9761B0027022316490993582206
:102F900020460CF051FB002313490296021D09AE96
:102FA0000591CDE903330321D2B20197009318466E
:102FB00006960EF0EFF831460FF072FB38B9256136
:102FC00000200BB0F0BDFBD2AF1B0026DCE70C20CD
:102FD0000BB0F0BDAFF300808D49FD1A0700000073
:102FE00000CA9A3BC8770020C91502000000000003
:102FF00070B5294C9DF810E094F8565015F0020574
:1030000042D110F0080F4FEA500605D094F8AEC038
:103010001CF0020F38D1583471B3A4F844104FEAB1
:10302000401C94F832101D484FEACE0E0EF0180ED8
:103030000CF0200C4CEA0E0C21F038014CEA010C8B
:1030400094F83C1084F832C066F3020184F83C1016
:1030500094F8561063F3830184F85610A2FB000322
:10306000912101FB02310AA3D3E90023FDF760FFA0
:10307000A064E064284670BD94F83C3061F302031C
:1030800084F83C30284670BD0C25284670BD00BF32
:103090008D49FD1A0700000060780020002AE784AF
:1030A00010B504469DF8080022854FEA411CC00077
:1030B000A17D00F018000CF0200C4CEA000C0C482C
:1030C00021F038014CEA010CA3FB0002912184F8A5
:1030D00016C001FB032104A3D3E90023FDF728FF59
:1030E000E06210BDAFF300808D49FD1A07000000BB
:1030F000002AE784000000002DE9F04F90F85630D8
:1031000090F83220DFF85492DFF854826FF3000316
:10311000044600F13E01C3F3800060F386128DB0D7
:1031200084F8563084F832200EF0D2F994F8322028
:10313000B4F844308448E46102F07902002684F84F
:1031400032209121A3FB000201FB0321C4E90566A3
:103150007BA3D3E900232670FDF7EAFE7B4AE36CEC
:10316000A364A4EB0905A2FB05251833C5F3871555
:1031700031229842A26005EB450298BF0346666083
:10318000E6608CBF23612061074648F8223098BF73
:10319000A6644FEA450A002D5AD199F8943003F0FD
:1031A0000703032B72D84FF0000B0EF03BF9236A94
:1031B00000F11806002B00F083800DF12C09AA44C1
:1031C00008EB8A030993CDF820900694B4F84430B4
:1031D0005D484FF00008A3FB0002CDF80C80912160
:1031E00001FB032123690493594B0793594B059322
:1031F0004FF0020A52A3D3E90023CDF82CA0FDF72B
:1032000097FE104619464FF47A720023FDF790FEA0
:1032100006355E44EDB2CDE90170032133462A46FE
:10322000CDF8008040460DF055FF49460FF038FAC2
:10323000002841D194F8563043EA0A0384F8563006
:1032400014F05CFC002856D000200DB0BDE8F08FD3
:10325000012DA8D199F83C30DB07A4D5A66C002E2F
:10326000A1D0B9F8443038489121A3FB000201FBFA
:10327000032133A3D3E90023FDF75AFE87424FF021
:10328000000B47D00023C8F80C308EE7A66C002E48
:1032900089D0B9F89C302C489121A3FB000201FB96
:1032A000032127A3D3E90023FDF742FE874226D05E
:1032B0000023C8F8003076E70C200DB0BDE8F08F91
:1032C0000DF12C09CDE90A3321694B460AAA0320E6
:1032D00001F096FE00287FF472AF0B991E4818A3E8
:1032E000D3E90023A1FB0001FDF722FE0A9B20F099
:1032F0007F461E4463E750461FF0B2FBA4E7D9F8AF
:10330000A03033449F42D3D302339F429CBF193E27
:103310002661CDE7D9F8483033449F42B2D3023317
:103320009F42AFD8193E2661D9F84830C4F848B05A
:10333000C9F848B003F1020BA4E700BFAFF3008067
:103340008D49FD1A07000000002AE784A38B2EBADE
:10335000C9150200899E020000CA9A3B60780020CD
:1033600048780020000000002DE9F04F0B79082B71
:1033700093B00C46074600F0FA80092B00F0D0808D
:10338000062B11D0B24AB349B3484FF4CC7331F095
:1033900004F9002383F31188BFF36F8F03231846CA
:1033A00002DF13B0BDE8F08FD1F80890D9F81830DB
:1033B0006BB1A74AA949A848D92331F0EEF80023F8
:1033C00083F31188BFF36F8F0323184602DFD9F808
:1033D0000080404617F036F90630C3B20B93012047
:1033E000A37E2760002666F38613A37694F8213027
:1033F000E660002B74D004F1220A3546B64694F8F4
:103400002220910669D094F823C01CF0010F14BF4C
:1034100004F12A0104F124011CF0020F18BF063147
:103420001CF0040F18BF01311CF0080F18BF023147
:103430001CF0100B1CBF8B4603311CF0200F18BF73
:1034400012311CF0400F18BF0131C2F30502A1EB8D
:103450000A010132D2B2C9B28A4238BF0A469A4240
:103460003ABF9A1A5FFA82FA4FF0000ABBF1000FD6
:1034700000F0B9809BF802C09BF801104FEA0C22C3
:1034800002F4F8520A4300F0AE80BEF1000F40F0A3
:10349000F480BCF15F0F4FEA5C1E40F22181002DE9
:1034A00000F04F822B8F53449BB22B87A383B8F13C
:1034B000000F00F0AD8098F856306A6BDB0700F122
:1034C000FC80D460EE6A6C63002E00F0B080284669
:1034D00013B0BDE8F04F17F0D9B9013BDBB2CDB95D
:1034E000A383214638460FF02BF813B0BDE8F04F08
:1034F0000FF032B8082394F81AE0237100227346C3
:1035000062F38613A37694F821302760E260002BE3
:1035100040F090822A8F13449BB22B87A383C6E787
:103520008E684F4B35689D423ED1D5F82C90B9F14D
:10353000000F00F0C6804A493C2208460CF07CF897
:103540000830C3B20B93D9F8000017F095F8804605
:10355000707900F00700022878D00428CAD001282A
:1035600054D03B4A3B493C484FF4AB730FE7D1F88A
:103570000890D9F818306BB1354A38493648EC23F1
:1035800031F00BF8002383F31188BFF36F8F03230F
:10359000184602DFD9F80080404617F053F806308D
:1035A000C3B20B9304201BE7D1F80C80B8F1000FD5
:1035B00000F0AC81D8F80050EB6A9E4258D0244A03
:1035C0002849254840F21D1330F0E7FF002383F31C
:1035D0001188BFF36F8F0323184602DFFF23B14624
:1035E0000B934646AFE7002D50D02B8F53449BB230
:1035F0002B87A383BEF1000F3FF459AF6B6B002BF9
:103600004AD0DC606C6313B0BDE8F08F062372E72C
:103610000F4A1549104840F2C13330F0BEFF88F31D
:103620001188BFF36F8F0323184602DF43E7084A70
:103630000E49094840F2E93330F0AFFF86F31188B4
:10364000BFF36F8F0323184602DF40E7072352E7DB
:10365000D4B5040054AB04007CAA040030B60400C6
:103660003C7900204CB60400CCB5040018B6040028
:10367000FF23B1460B93464665E7002D00F05581C8
:103680002B8F53449BB22B87A383B7E7A4F81CA0CE
:10369000BEF1000F3FF425AFAF4AB049B04840F249
:1036A0005A2330F07AFF002383F31188BFF36F8F22
:1036B0000323184602DF6B6BA3E76B6BA342A0D119
:1036C0006FE6A54AA749A64840F2051330F065FF0A
:1036D00089F31188BFF36F8F0323184602DF2AE7AF
:1036E0009BF900100029B4BF4FF496711E2110F011
:1036F000040F0C9101FB02F29BF8001000F01881FE
:10370000D800A37EC3F380035B002B30013300FAA3
:1037100003F303F5BC730C9803F5967C1018604511
:10372000C0F0F08049064CBF32214FF4FA718E4848
:1037300002FB01F1A0FB0101890C0D910121CDE9F2
:103740000E3201FA0EF3D8B2109320F0B7FB616984
:103750000F9A0E9B11902F390A44D31A0D9A1B1AF7
:1037600082489B1AA3FB000179A3D3E90023FDF74C
:10377000DFFB20F07F430E9394F91A30002B80F288
:10378000B680002D00F002812B8F53449BB21E2B7C
:103790002B8704D994F91A20002ABFF688AE6A6BE9
:1037A000002A00F00D81D4602B8F6C63A3839BF8FB
:1037B0000010109BB28801F03F0141EA032122F47E
:1037C000E76240F23F7322F007020B401343B380DD
:1037D00094F91A30002BC0F2F580B8F1000F00F018
:1037E000108198F8563013F001037FF466AF6B60D8
:1037F000EB603123AB60737903F00703032B00F216
:10380000A38003F10902D2005B10DA40119B5748F4
:1038100003F205331344564A0721E3FB0021104607
:103820004BA3D3E90023FDF783FB0D9B0C9A2F33A9
:1038300002EB430320F07F4028610022B3600221A5
:1038400001200BF069FF0B9AFF2A1BD023690E9908
:103850000026493B0B44CDE90066012130460DF0BE
:10386000B1FC10F0FD0F0DD03B4A42493C4840F2FC
:10387000963330F092FE86F31188BFF36F8F0323E7
:10388000184602DF3C493C2228460BF0D5FE3B4A55
:103890002369CDE907253A4ACDE9052529690024A0
:1038A000CDE9034100F108020E990091CDE90144F0
:1038B000493BD2B2012120460DF0D8FB10F0FD0F9C
:1038C0000DD0254A2F49264840F2A63330F065FE38
:1038D00084F31188BFF36F8F0323184602DF0122A0
:1038E0000221104613B0BDE8F04F0BF015BF0DF0EC
:1038F00099FD23690E9A383B99180DF095FD020247
:103900003FF53FAF002D7FF4D2ADEAE5124A1E49E4
:1039100013484FF48D7330F040FE88F31188BFF3E5
:103920006F8F0323184602DF44E6A4F81CA0B3E619
:1039300000F0030C63440933DB00C0F34000C340D4
:10394000E9E6A4F81CA0CCE54FF434725EE700BFB2
:103950008D49FD1A07000000D4B5040060B60400CC
:103960007CAA040040B6040083DE1B4300CA9A3BD5
:103970008C49FD1AA0B604003C79002079A9020008
:1039800075A70200D0B6040044B604002C480BF022
:1039900025FE0546002843D0002290F82010027032
:1039A000C0E9052262F3C7115346A0F838A0C061F0
:1039B00080F8201002634263C0F82C9000F11C06CE
:1039C0002C63F2E6D9F8183083B1B3420ED01D4A09
:1039D0001D491E4840F2333330F0DFFD002383F3EE
:1039E0001188BFF36F8F0323184602DFC9F81860F0
:1039F000A37E43F04003A37633796FF386133371CC
:103A0000CFE4104A1249114840F24A3330F0C5FD64
:103A100088F31188BFF36F8F0323184602DFE0E6B7
:103A200094F91A30002BBFF65CADA37E43F040033F
:103A3000A37656E5CEF3C00E04F1220ADFE400BF00
:103A400038790020D4B5040074B604007CAA0400C0
:103A5000CCB50400000000002DE9F04F05468BB006
:103A60008B46012002219946144624F0EDFD0022E8
:103A70000221824601200BF04FFE3F494FF4E072D5
:103A800028460BF0D9FD00F109063C4B0093F6B235
:103A900001954B463246012100200DF019FC10F033
:103AA000FD0F0ED0364A3749374840F68F0330F0C5
:103AB00074FD002383F31188BFF36F8F032318462F
:103AC00002DF324BA4FB0348204629A3D3E900239D
:103AD0004146FDF72DFA2E4B20F07F47A7FB03311F
:103AE0000722E01A02FB071168EB01014FF47A721A
:103AF0000023FDF71DFACDE90170CDF800B008955F
:103B00000695296995F9434022480491224931EAF2
:103B1000240128BF01460591204C07944FF6FE7101
:103B200003914B463246012100200DF09FFA10F020
:103B3000FD0F0ED0124A1349134840F6A40330F08B
:103B40002CFD002383F31188BFF36F8F03231846E6
:103B500002DFBAF1000F02D10BB0BDE8F08F0122F5
:103B6000022110460BB0BDE8F04F0BF0D5BD00BFF1
:103B70008D49FD1A0700000070100020D9AF020027
:103B800040B70400A0B604007CAA040000CA9A3B17
:103B90008D49FD1A5D1703006919030079AF020012
:103BA0002DE9F0418468228E4FF6FF739A428CB063
:103BB00045D0054620461AF071FD2B7D012B00F003
:103BC0002281022B00F01581002B00F0F48094F884
:103BD0006061002E40F010812B8A678F94F943209A
:103BE000CDE90A6673B3002AC0F25A810023A4F813
:103BF0009E31AA7C238FFD1802F003030135012BAF
:103C0000ADB23BD0B4F8A231002B00F005819D424B
:103C100080F059815B1B9BB20022062BA4F8A231D5
:103C2000628740F2F68094F943309342C0F25081AB
:103C3000002326E09DF82710204617F059FF0CB00E
:103C4000BDE8F081002AB8BF84F88961238FAA7C7F
:103C5000FD1802F003030135012BADB20ED0B4F80C
:103C60009E31002BCED0AB4240F23C815B1BA4F8CE
:103C70009E31B4F8A231002BC9D102E00023A4F890
:103C8000A23194F8482063F3820284F84820294640
:103C90000DF1270220461AF023FA7430CAD0B4F886
:103CA0009C312BB1AB4240F2EC805B1BA4F89C3101
:103CB000B4F898312BB1AB4240F2DA805B1BA4F828
:103CC0009831658F16B9AF4200F0C9800135ADB2A9
:103CD00094F8DD3013F0010731D1DDE90A130A460B
:103CE000002B40F0CC80002900F0BB801F46184616
:103CF000228EE4690694CDE9035609329A4D02906A
:103D0000CDE90017D2B20121002005950DF042FA4D
:103D100010F0FD0F93D00EF0EDFC84428FD0934A4B
:103D2000934994484FF4AE6330F037FC002383F39B
:103D30001188BFF36F8F0323184602DF7FE794F9E2
:103D400043206FF30003002A84F8DD307FDB94F812
:103D50008200C0F3C00100F0070020F0ADF8B4F815
:103D60007A20B4F878301344628D03F20933134497
:103D70000344814A81480721E3FB0021104678A3D0
:103D8000D3E90023FDF7D4F8DDE90A1320F07F42E0
:103D900020692261904235BF171A801A002000273F
:103DA0000A46002BA4D157EA010CA1D1002858D013
:103DB00019461F469CE794F89A3003F01803182B15
:103DC0007FF405AFA18EB4F89A218B1D9A42C4BF2F
:103DD000931F5B1AB4F89611CCBF9BB2134699425D
:103DE00000F09C80A4F89631A4F89831A4F89C21A6
:103DF000EDE63D2684F86061314620460CB0BDE812
:103E0000F04117F075BE0023A4F89C31A4F8983156
:103E1000DDE60126334634E7628E052A97BF01327C
:103E200040F2E2434FF4FA7392B203FB02F2B4F8A9
:103E3000A03142F2107101FB0323013BB3FBF2F30B
:103E40009BB2A4F8A231002B7FF4E1AE19E794F8FD
:103E50008300012100F0070020F030F87FE73546AD
:103E600036E7002D43D00027114638463B463FE752
